:020000040000FA
:040800002FEF0DF0D9
:08080800056ED8CF06F0E0CF29
:1008100007F00001E9CF0DF0EACF08F0E1CF09F0D1
:10082000E2CF0AF0D9CF0BF0DACF0CF0F3CF14F00F
:10083000F4CF15F0FACF16F000C00FF001C010F0A1
:1008400002C011F003C012F004C013F09DA02CEF01
:1008500004F09EB04CEF0BF0A0AA32EF04F0A1BA66
:1008600017EF0BF00FC000F010C001F011C002F044
:1008700012C003F013C004F00DC0E9FF08C0EAFF86
:10088000088E09C0E1FF0AC0E2FF0BC0D9FF0CC00F
:10089000DAFF14C0F3FF15C0F4FF16C0FAFF0550CD
:1008A00007C0E0FF06C0D8FF1000F76ABA0FF66E67
:1008B000080EF7220900F5501200040301000000A1
:1008C00000000000000000000000F76ADA0FF66E7A
:1008D000080EF7220900F550120004000100000084
:1008E00000000000000000000000F76AFA0FF66E3A
:1008F000080EF7220900F5501200400008004000E1
:1009000000000000000000000000000000000000E7
:100910000000000000000000000008AE03D0F2CF8D
:100920000EF0F29EF76A3C0FF66E090EF7220900F0
:10093000F55008AE02D00EBEF28E1200400000004C
:100940004000000000000000000000000000000067
:10095000000000000000000000000000F76A6C0FBB
:10096000F66E090EF7220900F55012000902430045
:10097000020100C032090400000102020100052446
:1009800000100104240202052406000105240100D0
:1009900001070581030800FA09040100020A0000AA
:1009A00000070502024000FA070582024000FA0033
:1009B000F76AC00FF66E090EF7220900F550120013
:1009C0000200F76AD20FF66E090EF7220900F55001
:1009D0001200120110010200004061043300000106
:1009E00001020001F76AF40FF66E090EF722090002
:1009F000F55012000403090408034D00500047009D
:100A00001E035000490043002000550053004200DF
:100A10002D00520053003200330032002000F2CF8C
:100A20000EF0F29EF76A380FF66E0A0EF7220900F2
:100A3000F5500EBEF28E1200280C0106F2CF0EF019
:100A4000F29EF76A560FF66E0A0EF7220900F5506D
:100A50000EBEF28E12000C00F2CF0EF0F29EF76A7C
:100A6000720FF66E0A0EF7220900F5500EBEF28ED6
:100A700012002D2041524553202D0000F2CF0EF0E0
:100A8000F29EF76A960FF66E0A0EF7220900F550ED
:100A90000EBEF28E120020452E502E532E20000046
:100AA0006D926994689422EF0BF06A6A68922BEF5A
:100AB0000BF02C6A2B6A250E2A6E800E296E2D6A89
:100AC0002E6A080E2F6E7F6B7A93316A306A7B6BC9
:100AD0007C917A81000CA96BA95101080AE3036A91
:100AE000A951270FE96E000E0320EA6EEF6AA92BC9
:100AF000F3D7DFDF1A6A010E1B6E196A000C010EB4
:100B0000B26FB2510F080EE3700EB225016E0F0ED8
:100B1000036ED8B0032A01C0E9FF03C0EAFFEF6A01
:100B2000B22BEFD71E6A1D6A000C400E0401016F44
:100B3000050E036F026B880E006F046B050E076FC6
:100B4000400E066F0001000C6A6A686A9F0E6B6EA9
:100B5000390E696E6E6ABFDFD2DF160E706E68A640
:100B600002D06896FCD76D98E0DF030E1F6E31EF60
:100B70000BF0698468986D8237EF0BF0689C3DEF4D
:100B80000BF070A002D0D1DF7090689A43EF0BF0A9
:100B9000ADC020F0000CFF0E206E000CAB6B265297
:100BA00035E0AB513F0832E31C5005E0020A0DE08E
:100BB000010A15E01ED0036A2550F2CFADF0F29E77
:100BC000CDDEADBFF28EAC6F14D0036A2550F2CFEC
:100BD000ADF0F29E07DFADBFF28EAC6F0AD0036AB4
:100BE0002550F2CFADF0F29EECDEADBFF28EAC6FD1
:100BF00000D0252A2606AB51AB2B036A400FE96EC5
:100C0000050E0320EA6EACC0EFFFC9D7265204E1FF
:100C1000AB51400801E0196AABC0ADF0B9DF000C80
:100C2000256A1C6A05010351010A000105E0030A57
:100C300008E0010A09E01FD0120E266E030E1C6E9A
:100C40001CD0430E266E19D0020E1C6E036A0501DD
:100C50000251210FE96E000E0320EA6EEFCF25F05E
:100C6000036A2550F2CFAAF0F29E0001BBDEAABFB4
:100C7000F28E266E02D08FDF0CD00501075305E1FE
:100C80002650065D02E206C526F0010E196E00012F
:100C900085DF63EF07F0AA5304E1040E1F6E2FDF18
:100CA000C1D0050E1F6EAD6F800EAC6F010EAB6F25
:100CB000AB510F08D8A0B6D0AE6B036AAB51F2CFE0
:100CC000B2F0F29E02DEB2BFF28E000A51E0040ED4
:100CD000AE6FD890AB35036AF2CFB2F0F29E1DDE54
:100CE0000900F5CF03F0B2BFF28EAF6F03C0B0F0D2
:100CF000AB51080DF350010F016E040E036ED8B016
:100D0000032A01C0E9FF03C0EAFFAFC0EFFFAB5108
:100D1000080DF350020F016E040E036ED8B0032AC3
:100D200001C0E9FF03C0EAFFADC0ECFFED52ACC06B
:100D3000EFFFD890AB35036AF2CFB2F0F29EEDDD53
:100D40000900F5CF03F0B2BFF28EAC270350AD23FC
:100D5000880EB16FB0B1B181B0B3B183AB51080DA2
:100D6000F3CF01F0040E01C0E9FFEA6EB1C0EFFF5E
:100D7000036AAB51F2CFB2F0F29E97DDB2BFF28EB2
:100D8000000A31E0AE83AB51080DF350060F016E3F
:100D9000040E036ED8B0032A01C0E9FF03C0EAFFC6
:100DA000ADC0ECFFED52ACC0EFFFD890AB35036A9D
:100DB000F2CFB2F0F29E99DD0900F5CF03F0B2BF99
:100DC000F28EAC270350AD23AB51080DF350040F46
:100DD000016E040E036ED8B0032A01C0E9FF03C000
:100DE000EAFF400EEF6EAE51060802E10E0EAE6F46
:100DF000036AAB51F2CFB2F0F29E57DDB2BFF28E72
:100E0000020801E0AE89700EAB25016E0F0E036E75
:100E1000D8B0032A01C0E9FF03C0EAFFAEC0EFFF6C
:100E2000AB2B46D75DEF07F00501015100010DE046
:100E3000010A14E0020A1EE0060A27E0030A2CE079
:100E40000E0A2BE0010A2FE03CD01BC040F5050143
:100E5000416B020E0001AD6F9BDE35D00501022D06
:100E600006D0010E1B160001AD6B92DE02D0000110
:100E700092DE29D00501022D05D01B820001AD6B49
:100E800087DE02D0000187DE1ED0020E196E02C579
:100E900024F0AD6B7DDE17D0C3D61AC040F5010E2D
:100EA000AD6F76DE10D005010251010808E302C5DE
:100EB0001AF002C5AAF00001EED6AD6B69DE0001A2
:100EC00002D069DE00D0DBEF08F01AC0AAF00501FD
:100ED0000151000105E00A0A0BE0010A2BE03CD0B9
:100EE0000501406B416B020E0001AD6F51DE36D043
:100EF000AA531EE0010EAA5D036AF2CFACF0F29E87
:100F000057DDACBFF28E016E0501045DD8A002D0A2
:100F100000010ED0036A0451270FE96E000E032072
:100F2000EA6EEFCF40F5010E0001AD6F31DE01D06A
:100F300032DE14D0AA530EE0036A05010451270FD4
:100F4000E96E000E0320EA6E02C5EFFF0001AD6BF3
:100F50001FDE01D020DE02D01EDE00D0DBEF08F065
:100F6000AB91AABFAB81AA9FABA110D0036AAA51D3
:100F7000F2CFACF0F29E99DCACBFF28E000A02E137
:100F8000000E01D0010E016E10D00FD0036AAA51DD
:100F9000F2CFACF0F29E99DCACBFF28E000A02E117
:100FA000000E01D0010E016E00D047EF08F0AB91AA
:100FB000AABFAB81AA9FABA110D0AA51080DF350D4
:100FC000040F016E040E036ED8B0032A01C0E9FFBE
:100FD00003C0EAFF880EEF6E09D0AA51080DF3CFC7
:100FE00001F0040E01C0E9FFEA6EEF6A56EF08F067
:100FF000AB91AABFAB81AA9FABA110D0AA51080D9B
:10100000F350040F016E040E036ED8B0032A01C022
:10101000E9FF03C0EAFF840EEF6E0AD0AA51080D63
:10102000F3CF01F0040E01C0E9FFEA6E840EEF6E0B
:101030005CEF08F0AB91AABFAB81AA9FABA110D027
:10104000AA51080DF350040F016E040E036ED8B0C0
:10105000032A01C0E9FF03C0EAFFEFCFACF00AD0DA
:10106000AA51080DF3CF01F0040E01C0E9FFEA6EAA
:10107000EFCFACF0ACAF02D0ACB502D0000E01D0D7
:10108000010E016E66EF08F004C5AAF069D701529F
:1010900029E005010151010A000105E0020A09E009
:1010A000030A0DE01DD004C5AAF081D7AD6B70DD39
:1010B00019D004C5AAF09CD7AD6B6ADD13D0050129
:1010C000406B416B04C5AAF00001B4D7015204E0A3
:1010D000010E0501406F0001020EAD6F59DD02D017
:1010E0005ADD00D0DBEF08F0FE0E206E000C05018B
:1010F000042D01D002D0045348E1015100010BE05E
:10110000010A0DE0210A1CE0010A1FE0030A2EE09B
:10111000010A31E037D0010E806FE6DF35D0050ED1
:10112000EA6E400EE96EE26A320EE16E080E016E62
:10113000E6CFEEFF012EFCD706C5ADF029DD24D0A9
:10114000020E806F7A83D0DF1FD0050EEA6E400E4C
:10115000E96EE26A290EE16E070E016EE6CFEEFF40
:10116000012EFCD7070EAD6F13DD0ED002C57FF048
:10117000AD6B0EDD09D002C531F003C530F0AD6BAB
:1011800007DD02D008DD00D005010001DBEF08F02B
:10119000196A050100517F0B000107E0010A06E012
:1011A000030A05E0230A04E004D03ED68ED66CD7AD
:1011B0009ED7F1DC00D0C2EF0AF0AA51080DF3CFA0
:1011C00001F0040E01C0E9FFEA6EEFCFACF0AB51C5
:1011D000020806E1ACAD02D0AB6B02D0010EAB6FE2
:1011E000AB51030812E1840EAC6FAA51080DF35005
:1011F000040F016E040E036ED8B0032A01C0E9FF8C
:1012000003C0EAFF840EEF6E09D0AB2D03D0C80EE9
:10121000AC6F04D0AB5302E1880EAC6F036A010ED1
:10122000026EAA51006E05E0D89002360336002EF9
:10123000FBD70250FF0A006EFF0E031A00501D1666
:1012400003501E16D890AA35036AF2CFAFF0F29E73
:101250008DEC04F00900F5CF03F0AFBFF28EAD6F57
:1012600003C0AEF0AA51080DF350010F016E040E39
:10127000036ED8B0032A01C0E9FF03C0EAFFADC086
:10128000EFFFAEB1AC81AEB3AC83AA51080DF3CF82
:1012900001F0040E01C0E9FFEA6EACC0EFFF000CE4
:1012A000B651080DF350040F016E040E036ED8B052
:1012B000032A01C0E9FF03C0EAFFEFCFBAF0BABFCB
:1012C0005BD0B651080DF350050F016E040E036E8E
:1012D000D8B0032A01C0E9FF03C0EAFFB7C0EFFF9F
:1012E000B951020816E1B651080DF350040F016E12
:1012F000040E036ED8B0032A01C0E9FF03C0EAFF61
:10130000EFCFBAF0BAAD02D0B96B02D0010EB96F0F
:1013100013D0B951040810E1B651080DF3CF01F014
:10132000040E01C0E9FFEA6EEFCFBAF0BAAD03D008
:10133000010EB96F01D0B96BB92D03D0C80EBA6FC9
:1013400004D0B95302E1880EBA6FB8B1BA81B8B30C
:10135000BA83B651080DF350040F016E040E036EEC
:10136000D8B0032A01C0E9FF03C0EAFFBAC0EFFF0B
:10137000010E016E03D000D0000E016E000C8051F2
:10138000010A03E0030A12E022D0EA6A320EE96E93
:10139000050EE26EE16A080E016EE6CFEEFF012E49
:1013A000FCD7AD6BC8EC05F0806B15D0EA6A290E4E
:1013B000E96E050EE26EE16A070E016EE6CFEEFF02
:1013C000012EFCD7806BAD6BC8EC05F004D0806BB0
:1013D00095EC05F000D00DEF0AF0AB51080DF3507D
:1013E000010F016E040E036ED8B0032A01C0E9FF9D
:1013F00003C0EAFF036AEFCF01F003C002F006EF7B
:101400000AF07C817E6B020EAB6FE7D701C07DF0E6
:1014100012EF0AF0AA5302E1B2D714D0AA5102087F
:1014200002E1EFD70FD0036A010E026EAA51006EDF
:1014300005E0D89002360336002EFBD702501D126D
:1014400003501E12000CABC06EFFAB5303E0040E42
:101450001F6E02D0020E1F6E33EF0AF01A6A196A6D
:1014600024C0ABF0F0D7ACEF0AF0AB51080DF3504D
:10147000040F016E040E036ED8B0032A01C0E9FF09
:1014800003C0EAFFEFCFB3F0B3BF3FD0AB51080DBD
:10149000F350060F016E040E036ED8B0032A01C08C
:1014A000E9FF03C0EAFFECCF03F0ED52EFCFB4F059
:1014B00003C0B5F0B26BB16BB251AF5D1AE303E19B
:1014C000AE51B15D16E2ACC0E9FFADC0EAFFEFCFAF
:1014D000B8F0B5C0EAFFB4C0E9FFB8C0EFFFB42B65
:1014E000D8B4B52BAC2BD8B4AD2BB12BD8B4B22B10
:1014F000E3D7ABC0B6F0AFC0B8F0AEC0B7F0B0C085
:10150000B9F0CEDE015003D000D0000E016E97EF8F
:101510000AF07B530DE07A91020EAB6FAD6B3A0E81
:10152000AC6FAF6B7BC0AEF0020EB06F9ED77B6B23
:101530009DEF0AF07B5302E0ECD701D07A81B1EF46
:101540000AF0AA530AE1192C03D0CEEC05F004D01E
:101550001950020801E182D704D0AA51020801E122
:10156000E9D7000C6C30A96FA933A9331F0EA91756
:101570006C523BE1040100513C0B34081BE1046B4D
:10158000000106D6203C05D0AA6B030EAB6F15DE1A
:101590000ED0AA6B020EAB6F10DE2050FE0807E0E3
:1015A000B66BB86B20C0B7F0040EB96F79DE6D98DA
:1015B00019D0040100513C0B040815E10001AA6B8D
:1015C00029DFAA6B020EAB6FF8DD2050FE080AE09F
:1015D000203C01D007D0B66BB86B20C0B7F0010E2D
:1015E000B96F5EDE040120D000016C50040812E1E6
:1015F000FF0E206EAA6BA5DF203C01D008D0B66B91
:10160000B86B20C0B7F0020EB96F4ADE02D095EC7D
:1016100005F009D06CB404D0A9C0AAF0FBDE03D059
:10162000A9C0AAF08EDF0401000148EF0BF01F52A1
:1016300001E12FD068522DE068A404D069A402D043
:1016400050EF05F06DA201D024D068A204D069A2A9
:1016500002D055EF05F068A004D069A002D0A4EF35
:1016600005F068A804D069A802D0B9EF05F068AC0D
:1016700004D069AC02D0BEEF05F068AA04D069AA14
:1016800002D0C1EF05F068A604D069A602D06AD7DF
:101690006896A19A32EF04F098B54BD0975304E1C5
:1016A0007AA502D092908980972D04D07AA702D093
:1016B000929289829751020804E17AA902D0929409
:1016C00089849751030804E17AAB02D09296898607
:1016D0009751040804E17AAD02D0929A898A975111
:1016E000050804E17AAF02D096908D8097510608E4
:1016F00004E198A102D096928D829751070804E1E7
:1017000098A302D096948D84D8909735036A870F5A
:10171000E96E000E0320EA6EECCF03F0ED52EF50BD
:10172000FF08996FFF0E03549A6F9AC0CFFF99C0BC
:10173000CEFF98A550D0975304E17AA502D092909D
:101740008990972D04D07AA702D0929289929751CE
:10175000020804E17AA902D092948994975103086F
:1017600004E17AAB02D0929689969751040804E17D
:101770007AAD02D0929A899A9751050804E17AAF1E
:1017800002D096908D909751060804E198A102D05E
:1017900096928D929751070804E198A302D09694EF
:1017A0008D94D8909735036A870FE96E000E032059
:1017B000EA6EECCF03F0ED52EF50B30F996FE20EEB
:1017C00003209A6F9AC0CFFF99C0CEFF972B9751F5
:1017D0000708D8A0976B98759E9032EF04F06D6A59
:1017E000696A080E6F6E94503009946E1F6A186A09
:1017F000F2BE188EF29E6BEC05F018BEF28E1E6AD9
:101800001D6A26EF0CF0186AF2BE188EF29E6BEC81
:1018100005F018BEF28E6D6A140E6F6E696A6D86E1
:10182000010E1F6E17EF0CF06DB601D0ECD71F2C18
:101830000BD06DBA09D0686A696AA08AC00EF2122C
:10184000110E696E020E1F6E000CC9D7EDDF1F501E
:101850000208FCE182EF0DF0EA6AA00EE96EEF509B
:101860000EE00F0E016E006A002EFED7012EFBD790
:101870008F0E006E002EFED70000EF2EF2D7000C68
:10188000A7B102D08A9601D08A869396A7B302D0D8
:101890008A9A01D08A8A939AA7B502D08A9E01D0EB
:1018A0008A8E939EA7B702D08A9C01D08A8C939C83
:1018B0000000959C8C8C070E006E002EFED700D089
:1018C000959C8C9C000CA86B959C8C8C000093863E
:1018D000A89181B6A881938AA89381BAA883938E90
:1018E000A89581BEA885938CA89781BCA887959C54
:1018F0008C9CA8C001F0000C93948A840000E3DF64
:1019000001C0A7F0E0DF01C0A6F0A739006EF00E1D
:1019100000160050A611016E91EF0CF0959E8C9E62
:10192000EBD701C0A6F001BEFBD7A45303E0959E00
:101930008C8E02D0959E8C9E000093948A94000019
:10194000959C8C9CA539A66F0F0EA617A6C0A7F074
:1019500097DFA5510F0BA66FA76F92DF000C959E26
:101960008C9E93948A94959C8C9C0F0EA06F74DF30
:101970009E6B9E51020808E3030EA76F81DF050EE0
:10198000A06F6ADF9E2BF5D7020EA76F79DF9E6BE3
:101990009E5103080FE3036A9E51F2CF9FF0F29E1F
:1019A0000FEC05F09FBFF28EA06FA46BA56FB6DFA2
:1019B0009E2BEED788EF0DF0A12D01D003D0400E65
:1019C000A26F01D0A26B010EA05DA227A2518009D7
:1019D000A36FA46BA56FA2DF000C9F510C0A05E05A
:1019E000060A0BE0020A0FE013D0A46B010EA56FEC
:1019F00095DF020EA06F30DF11D0010EA06F020E36
:101A0000A16FDADF0BD0A46B100EA56F87DF06D0B5
:101A1000010EA46F9FC0A5F081DF00D0000C7CB147
:101A200001D0FDD77E517E2B036A880FE96E050E2B
:101A30000320EA6EEFCF9EF07D517E5D0CE37C913A
:101A4000186AF2BE188EF29E020EAA6FAB6FDDEC22
:101A500008F018BEF28E9EC001F0BBEF0DF0F86AE0
:101A6000D09E088EEA6AE96AC150C00B0F09C16EA8
:101A7000070EB46E1F6A216A040E226E0C0E236ECE
:101A8000266A7B6B806B816B826BD00E876F070E33
:101A9000886FD00E896F070E8A6FB80E8B6F0B0E92
:101AA0008C6FA00E8D6F0F0E8E6F880E8F6F130EC2
:101AB000906F700E916F170E926F700E936F170EDE
:101AC000946F956B966B976B7A957A977A997A9BC8
:101AD0007A9D7A9F989198939895B30E996FE20E9C
:101AE0009A6F080E9C6F9D6BF29CF29EF2BEFDD722
:101AF000A50ECD6E9AC0CFFF99C0CEFF9D8059EC48
:101B000005F0A3D6C00EF212320EA06FA5DE27D7C5
:101B10009E6B9E511EEC05F0000904E09E2B9F6F0A
:101B20005CDFF7D7010EA06FA16F46DF9E6B9E5161
:101B30002CEC05F0000904E09E2B9F6F4EDFF7D7D9
:101B4000010EA06F020EA16F37DF9E6B9E513EEC1F
:101B500005F0000904E09E2B9F6F3FDFF7D77AB3B3
:101B600001D0FDD761DE1A52D8B4F5EF22F07CA186
:101B7000F5EF22F054D701C09BF09B51010AD8B475
:101B8000F8D3030AD8B4FAD3010AD8B4FDD3070AAC
:101B9000D8B4CAEF11F0010AD8B4D0EF11F0030A9B
:101BA000D8B4D6EF11F0010AD8B4DCEF11F00F0A67
:101BB000D8B4E2EF11F0010AD8B4E8EF11F0030A4B
:101BC000D8B4EAEF11F0010AD8B4FBEF11F0070A1C
:101BD000D8B40CEF12F0010AD8B41DEF12F0030ACA
:101BE000D8B42EEF12F0010AD8B43FEF12F01F0A5A
:101BF000D8B450EF12F0010AD8B461EF12F0030A22
:101C0000D8B473EF12F0010AD8B485EF12F0070AC6
:101C1000D8B497EF12F0010AD8B4A9EF12F0030A72
:101C2000D8B4BBEF12F0010AD8B4CDEF12F00F0A0E
:101C3000D8B4DFEF12F0010AD8B4F1EF12F0030AC2
:101C4000D8B403EF13F0010AD8B415EF13F0070A64
:101C5000D8B427EF13F0010AD8B439EF13F0030A10
:101C6000D8B44BEF13F0010AD8B45DEF13F03F0A7C
:101C7000D8B46FEF13F0010AD8B481EF13F0030A60
:101C8000D8B493EF13F0010AD8B4A5EF13F0070A04
:101C9000D8B4B7EF13F0010AD8B4C9EF13F0030AB0
:101CA000D8B4DBEF13F0010AD8B4EDEF13F00F0A4C
:101CB000D8B4FFEF13F0010AD8B411EF14F0030AFF
:101CC000D8B423EF14F0010AD8B435EF14F0070AA2
:101CD000D8B447EF14F0010AD8B459EF14F0030A4E
:101CE000D8B46BEF14F0010AD8B47DEF14F01F0ADA
:101CF000D8B48FEF14F0010AD8B4A1EF14F0030A9E
:101D0000D8B4B3EF14F0010AD8B4C5EF14F0070A41
:101D1000D8B4D7EF14F0010AD8B4E9EF14F0030AED
:101D2000D8B4FBEF14F0010AD8B40DEF15F00F0A88
:101D3000D8B41FEF15F0010AD8B431EF15F0030A3B
:101D4000D8B443EF15F0010AD8B455EF15F0070ADF
:101D5000D8B467EF15F0010AD8B479EF15F0030A8B
:101D6000D8B48BEF15F0010AD8B49DEF15F07F0AB7
:101D7000D8B4AFEF15F0010AD8B4C1EF15F0030ADB
:101D8000D8B4D3EF15F0010AD8B4E5EF15F0070A7F
:101D9000D8B4F7EF15F0010AD8B409EF16F0030A2A
:101DA000D8B41BEF16F0010AD8B42DEF16F00F0AC5
:101DB000D8B43FEF16F0010AD8B451EF16F0030A79
:101DC000D8B463EF16F0010AD8B475EF16F0070A1D
:101DD000D8B487EF16F0010AD8B499EF16F0030AC9
:101DE000D8B4ABEF16F0010AD8B4BDEF16F01F0A55
:101DF000D8B4CFEF16F0010AD8B4E1EF16F0030A19
:101E0000D8B4F3EF16F0010AD8B405EF17F0070ABB
:101E1000D8B417EF17F0010AD8B429EF17F0030A66
:101E2000D8B43BEF17F0010AD8B44DEF17F00F0A02
:101E3000D8B45FEF17F0010AD8B471EF17F0030AB6
:101E4000D8B483EF17F0010AD8B495EF17F0070A5A
:101E5000D8B4A7EF17F0010AD8B4B9EF17F0030A06
:101E6000D8B4CBEF17F0010AD8B4DDEF17F03F0A72
:101E7000D8B4EFEF17F0010AD8B401EF18F0030A55
:101E8000D8B413EF18F0010AD8B425EF18F0070AF8
:101E9000D8B437EF18F0010AD8B449EF18F0030AA4
:101EA000D8B45BEF18F0010AD8B46DEF18F00F0A40
:101EB000D8B47FEF18F0010AD8B491EF18F0030AF4
:101EC000D8B4A3EF18F0010AD8B4B5EF18F0070A98
:101ED000D8B4C7EF18F0010AD8B4D9EF18F0030A44
:101EE000D8B4EBEF18F0010AD8B4FDEF18F01F0AD0
:101EF000D8B40FEF19F0010AD8B421EF19F0030A92
:101F0000D8B433EF19F0010AD8B445EF19F0070A35
:101F1000D8B457EF19F0010AD8B469EF19F0030AE1
:101F2000D8B47BEF19F0010AD8B48DEF19F00F0A7D
:101F3000D8B49FEF19F0010AD8B4B1EF19F0030A31
:101F4000D8B4C3EF19F0010AD8B4D5EF19F0070AD5
:101F5000D8B4E7EF19F0010AD8B4F9EF19F0030A81
:101F6000D8B40BEF1AF0010AD8B41DEF1AF0FF0A2B
:101F7000D8B42FEF1AF0010AD8B441EF1AF0030ACF
:101F8000D8B453EF1AF0010AD8B465EF1AF0070A73
:101F9000D8B477EF1AF0010AD8B489EF1AF0030A1F
:101FA000D8B49BEF1AF0010AD8B4ADEF1AF00F0ABB
:101FB000D8B4BFEF1AF0010AD8B4D0EF1AF0030A70
:101FC000D8B4E2EF1AF0010AD8B4F4EF1AF0070A15
:101FD000D8B406EF1BF0010AD8B418EF1BF0030ABF
:101FE000D8B42AEF1BF0010AD8B43CEF1BF01F0A4B
:101FF000D8B44EEF1BF0010AD8B460EF1BF0030A0F
:10200000D8B472EF1BF0010AD8B484EF1BF0070AB2
:10201000D8B496EF1BF0010AD8B4A8EF1BF0030A5E
:10202000D8B4BAEF1BF0010AD8B4CCEF1BF00F0AFA
:10203000D8B4DEEF1BF0010AD8B4F0EF1BF0030AAE
:10204000D8B402EF1CF0010AD8B414EF1CF0070A50
:10205000D8B426EF1CF0010AD8B438EF1CF0030AFC
:10206000D8B44AEF1CF0010AD8B45CEF1CF03F0A68
:10207000D8B46EEF1CF0010AD8B480EF1CF0030A4C
:10208000D8B492EF1CF0010AD8B4A4EF1CF0070AF0
:10209000D8B4B6EF1CF0010AD8B4C8EF1CF0030A9C
:1020A000D8B4DAEF1CF0010AD8B4ECEF1CF00F0A38
:1020B000D8B4FEEF1CF0010AD8B410EF1DF0030AEB
:1020C000D8B422EF1DF0010AD8B434EF1DF0070A8E
:1020D000D8B446EF1DF0010AD8B458EF1DF0030A3A
:1020E000D8B46AEF1DF0010AD8B47CEF1DF01F0AC6
:1020F000D8B48EEF1DF0010AD8B4A0EF1DF0030A8A
:10210000D8B4B2EF1DF0010AD8B4C4EF1DF0070A2D
:10211000D8B4D6EF1DF0010AD8B4E8EF1DF0030AD9
:10212000D8B4FAEF1DF0010AD8B40CEF1EF00F0A74
:10213000D8B41EEF1EF0010AD8B430EF1EF0030A27
:10214000D8B442EF1EF0010AD8B454EF1EF0070ACB
:10215000D8B466EF1EF0010AD8B478EF1EF0030A77
:10216000D8B48AEF1EF0010AD8B49CEF1EF07F0AA3
:10217000D8B4AEEF1EF0010AD8B4C0EF1EF0030AC7
:10218000D8B4D2EF1EF0010AD8B4E4EF1EF0070A6B
:10219000D8B4F6EF1EF0010AD8B408EF1FF0030A16
:1021A000D8B41AEF1FF0010AD8B42CEF1FF00F0AB1
:1021B000D8B43DEF1FF0010AD8B44EEF1FF0030A68
:1021C000D8B45FEF1FF0010AD8B470EF1FF0070A10
:1021D000D8B481EF1FF0010AD8B492EF1FF0030AC0
:1021E000D8B4A3EF1FF0010AD8B4B4EF1FF01F0A50
:1021F000D8B4C5EF1FF0010AD8B4D6EF1FF0030A18
:10220000D8B4E7EF1FF0010AD8B4F8EF1FF0070ABF
:10221000D8B409EF20F0010AD8B41AEF20F0030A6D
:10222000D8B42BEF20F0010AD8B43CEF20F00F0A0D
:10223000D8B44DEF20F0010AD8B45EEF20F0030AC5
:10224000D8B46FEF20F0010AD8B480EF20F0070A6D
:10225000D8B491EF20F0010AD8B4A2EF20F0030A1D
:10226000D8B4B3EF20F0010AD8B4C4EF20F03F0A8D
:10227000D8B4D5EF20F0010AD8B4E6EF20F0030A75
:10228000D8B4F7EF20F0010AD8B408EF21F0070A1C
:10229000D8B419EF21F0010AD8B42AEF21F0030ACB
:1022A000D8B43BEF21F0010AD8B44CEF21F00F0A6B
:1022B000D8B45DEF21F0010AD8B46EEF21F0030A23
:1022C000D8B47FEF21F0010AD8B490EF21F0070ACB
:1022D000D8B4A1EF21F0010AD8B4B2EF21F0030A7B
:1022E000D8B4C3EF21F0010AD8B4D4EF21F01F0A0B
:1022F000D8B4E5EF21F0010AD8B4F6EF21F0030AD3
:10230000D8B407EF22F0010AD8B418EF22F0070A78
:10231000D8B429EF22F0010AD8B43AEF22F0030A28
:10232000D8B44BEF22F0010AD8B45CEF22F00F0AC8
:10233000D8B46DEF22F0010AD8B47EEF22F0030A80
:10234000D8B48FEF22F0010AD8B4A0EF22F0070A28
:10235000D8B4B1EF22F0010AD8B4C2EF22F0030AD8
:10236000D8B4D3EF22F0010AD8B4E4EF22F0F5EFAD
:1023700022F09D6B9C6B7A85F5EF22F09D6B010E30
:102380009C6F7A87F5EF22F09D6B020E9C6F7A8925
:10239000F5EF22F09D6B030E9C6F7A8BF5EF22F028
:1023A0009D6B040E9C6F7A8DF5EF22F09D6B050EF0
:1023B0009C6F7A8FF5EF22F09D6B060E9C6F9881D3
:1023C000F5EF22F09D6B070E9C6F9883F5EF22F0DE
:1023D000F5EF22F0D8909C35026E9D35036E0250C9
:1023E000870FE96E000E0320EA6EEC6AED523C0E98
:1023F000EF6EF5EF22F0D8909C35026E9D35036E9E
:102400000250870FE96E000E0320EA6EEC6AED526F
:102410005A0EEF6EF5EF22F0D8909C35026E9D3586
:10242000036E0250870FE96E000E0320EA6EEC6A1D
:10243000ED52780EEF6EF5EF22F0D8909C35026EDB
:102440009D35036E0250870FE96E000E0320EA6E81
:10245000EC6AED52960EEF6EF5EF22F0D8909C35B7
:10246000026E9D35036E0250870FE96E000E032049
:10247000EA6EEC6AED52B40EEF6EF5EF22F0D890F2
:102480009C35026E9D35036E0250870FE96E000E7B
:102490000320EA6EEC6AED52D20EEF6EF5EF22F0F9
:1024A000D8909C35026E9D35036E0250870FE96E01
:1024B000000E0320EA6EEC6AED52F00EEF6EF5EFBF
:1024C00022F0D8909C35026E9D35036E0250870F26
:1024D000E96E000E0320EA6E010EEC6EED520E0E58
:1024E000EF6EF5EF22F0D8909C35026E9D35036EAD
:1024F0000250870FE96E000E0320EA6E010EEC6EAB
:10250000ED522C0EEF6EF5EF22F0D8909C35026E56
:102510009D35036E0250870FE96E000E0320EA6EB0
:10252000010EEC6EED524A0EEF6EF5EF22F0D890F0
:102530009C35026E9D35036E0250870FE96E000ECA
:102540000320EA6E010EEC6EED52680EEF6EF5EFB1
:1025500022F0D8909C35026E9D35036E0250870F95
:10256000E96E000E0320EA6E010EEC6EED52860E4F
:10257000EF6EF5EF22F0D8909C35026E9D35036E1C
:102580000250870FE96E000E0320EA6E010EEC6E1A
:10259000ED52A40EEF6EF5EF22F0D8909C35026E4E
:1025A0009D35036E0250870FE96E000E0320EA6E20
:1025B000010EEC6EED52C20EEF6EF5EF22F0D890E8
:1025C0009C35026E9D35036E0250870FE96E000E3A
:1025D0000320EA6E010EEC6EED52E00EEF6EF5EFA9
:1025E00022F0D8909C35026E9D35036E0250870F05
:1025F000E96E000E0320EA6E010EEC6EED52FE0E47
:10260000EF6EF5EF22F0D8909C35026E9D35036E8B
:102610000250870FE96E000E0320EA6E020EEC6E88
:10262000ED521C0EEF6EF5EF22F0D8909C35026E45
:102630009D35036E0250870FE96E000E0320EA6E8F
:10264000020EEC6EED523A0EEF6EF5EF22F0D890DE
:102650009C35026E9D35036E0250870FE96E000EA9
:102660000320EA6E020EEC6EED52580EEF6EF5EF9F
:1026700022F0D8909C35026E9D35036E0250870F74
:10268000E96E000E0320EA6E020EEC6EED52760E3D
:10269000EF6EF5EF22F0D8909C35026E9D35036EFB
:1026A0000250870FE96E000E0320EA6E020EEC6EF8
:1026B000ED52940EEF6EF5EF22F0D8909C35026E3D
:1026C0009D35036E0250870FE96E000E0320EA6EFF
:1026D000020EEC6EED52B20EEF6EF5EF22F0D890D6
:1026E0009C35026E9D35036E0250870FE96E000E19
:1026F0000320EA6E020EEC6EED52D00EEF6EF5EF97
:1027000022F0D8909C35026E9D35036E0250870FE3
:10271000E96E000E0320EA6E020EEC6EED52EE0E34
:10272000EF6EF5EF22F0D8909C35026E9D35036E6A
:102730000250870FE96E000E0320EA6E030EEC6E66
:10274000ED520C0EEF6EF5EF22F0D8909C35026E34
:102750009D35036E0250870FE96E000E0320EA6E6E
:10276000030EEC6EED522A0EEF6EF5EF22F0D890CC
:102770009C35026E9D35036E0250870FE96E000E88
:102780000320EA6E030EEC6EED52480EEF6EF5EF8D
:1027900022F0D8909C35026E9D35036E0250870F53
:1027A000E96E000E0320EA6E030EEC6EED52660E2B
:1027B000EF6EF5EF22F0D8909C35026E9D35036EDA
:1027C0000250870FE96E000E0320EA6E030EEC6ED6
:1027D000ED52840EEF6EF5EF22F0D8909C35026E2C
:1027E0009D35036E0250870FE96E000E0320EA6EDE
:1027F000030EEC6EED52A20EEF6EF5EF22F0D890C4
:102800009C35026E9D35036E0250870FE96E000EF7
:102810000320EA6E030EEC6EED52C00EEF6EF5EF84
:1028200022F0D8909C35026E9D35036E0250870FC2
:10283000E96E000E0320EA6E030EEC6EED52DE0E22
:10284000EF6EF5EF22F0D8909C35026E9D35036E49
:102850000250870FE96E000E0320EA6E030EEC6E45
:10286000ED52FC0EEF6EF5EF22F0D8909C35026E23
:102870009D35036E0250870FE96E000E0320EA6E4D
:10288000040EEC6EED521A0EEF6EF5EF22F0D890BA
:102890009C35026E9D35036E0250870FE96E000E67
:1028A0000320EA6E040EEC6EED52380EEF6EF5EF7B
:1028B00022F0D8909C35026E9D35036E0250870F32
:1028C000E96E000E0320EA6E040EEC6EED52560E19
:1028D000EF6EF5EF22F0D8909C35026E9D35036EB9
:1028E0000250870FE96E000E0320EA6E040EEC6EB4
:1028F000ED52740EEF6EF5EF22F0D8909C35026E1B
:102900009D35036E0250870FE96E000E0320EA6EBC
:10291000040EEC6EED52920EEF6EF5EF22F0D890B1
:102920009C35026E9D35036E0250870FE96E000ED6
:102930000320EA6E040EEC6EED52B00EEF6EF5EF72
:1029400022F0D8909C35026E9D35036E0250870FA1
:10295000E96E000E0320EA6E040EEC6EED52CE0E10
:10296000EF6EF5EF22F0D8909C35026E9D35036E28
:102970000250870FE96E000E0320EA6E040EEC6E23
:10298000ED52EC0EEF6EF5EF22F0D8909C35026E12
:102990009D35036E0250870FE96E000E0320EA6E2C
:1029A000050EEC6EED520A0EEF6EF5EF22F0D890A8
:1029B0009C35026E9D35036E0250870FE96E000E46
:1029C0000320EA6E050EEC6EED52280EEF6EF5EF69
:1029D00022F0D8909C35026E9D35036E0250870F11
:1029E000E96E000E0320EA6E050EEC6EED52460E07
:1029F000EF6EF5EF22F0D8909C35026E9D35036E98
:102A00000250870FE96E000E0320EA6E050EEC6E91
:102A1000ED52640EEF6EF5EF22F0D8909C35026E09
:102A20009D35036E0250870FE96E000E0320EA6E9B
:102A3000050EEC6EED52820EEF6EF5EF22F0D8909F
:102A40009C35026E9D35036E0250870FE96E000EB5
:102A50000320EA6E050EEC6EED52A00EEF6EF5EF60
:102A600022F0D8909C35026E9D35036E0250870F80
:102A7000E96E000E0320EA6E050EEC6EED52BE0EFE
:102A8000EF6EF5EF22F0D8909C35026E9D35036E07
:102A90000250870FE96E000E0320EA6E050EEC6E01
:102AA000ED52DC0EEF6EF5EF22F0D8909C35026E01
:102AB0009D35036E0250870FE96E000E0320EA6E0B
:102AC000050EEC6EED52FA0EEF6EF5EF22F0D89097
:102AD0009C35026E9D35036E0250870FE96E000E25
:102AE0000320EA6E060EEC6EED52180EEF6EF5EF57
:102AF00022F0D8909C35026E9D35036E0250870FF0
:102B0000E96E000E0320EA6E060EEC6EED52360EF4
:102B1000EF6EF5EF22F0D8909C35026E9D35036E76
:102B20000250870FE96E000E0320EA6E060EEC6E6F
:102B3000ED52540EEF6EF5EF22F0D8909C35026EF8
:102B40009D35036E0250870FE96E000E0320EA6E7A
:102B5000060EEC6EED52720EEF6EF5EF22F0D8908D
:102B60009C35026E9D35036E0250870FE96E000E94
:102B70000320EA6E060EEC6EED52900EEF6EF5EF4E
:102B800022F0D8909C35026E9D35036E0250870F5F
:102B9000E96E000E0320EA6E060EEC6EED52AE0EEC
:102BA000EF6EF5EF22F0D8909C35026E9D35036EE6
:102BB0000250870FE96E000E0320EA6E060EEC6EDF
:102BC000ED52CC0EEF6EF5EF22F0D8909C35026EF0
:102BD0009D35036E0250870FE96E000E0320EA6EEA
:102BE000060EEC6EED52EA0EEF6EF5EF22F0D89085
:102BF0009C35026E9D35036E0250870FE96E000E04
:102C00000320EA6E070EEC6EED52080EEF6EF5EF44
:102C100022F0D8909C35026E9D35036E0250870FCE
:102C2000E96E000E0320EA6E070EEC6EED52260EE2
:102C3000EF6EF5EF22F0D8909C35026E9D35036E55
:102C40000250870FE96E000E0320EA6E070EEC6E4D
:102C5000ED52440EEF6EF5EF22F0D8909C35026EE7
:102C60009D35036E0250870FE96E000E0320EA6E59
:102C7000070EEC6EED52620EEF6EF5EF22F0D8907B
:102C80009C35026E9D35036E0250870FE96E000E73
:102C90000320EA6E070EEC6EED52800EEF6EF5EF3C
:102CA00022F0D8909C35026E9D35036E0250870F3E
:102CB000E96E000E0320EA6E070EEC6EED529E0EDA
:102CC000EF6EF5EF22F0D8909C35026E9D35036EC5
:102CD0000250870FE96E000E0320EA6E070EEC6EBD
:102CE000ED52BC0EEF6EF5EF22F0D8909C35026EDF
:102CF0009D35036E0250870FE96E000E0320EA6EC9
:102D0000070EEC6EED52DA0EEF6EF5EF22F0D89072
:102D10009C35026E9D35036E0250870FE96E000EE2
:102D20000320EA6E070EEC6EED52F80EEF6EF5EF33
:102D300022F0D8909C35026E9D35036E0250870FAD
:102D4000E96E000E0320EA6E080EEC6EED52160ED0
:102D5000EF6EF5EF22F0D8909C35026E9D35036E34
:102D60000250870FE96E000E0320EA6E080EEC6E2B
:102D7000ED52340EEF6EF5EF22F0D8909C35026ED6
:102D80009D35036E0250870FE96E000E0320EA6E38
:102D9000080EEC6EED52520EEF6EF5EF22F0D89069
:102DA0009C35026E9D35036E0250870FE96E000E52
:102DB0000320EA6E080EEC6EED52700EEF6EF5EF2A
:102DC00022F0D8909C35026E9D35036E0250870F1D
:102DD000E96E000E0320EA6E080EEC6EED528E0EC8
:102DE000EF6EF5EF22F0D8909C35026E9D35036EA4
:102DF0000250870FE96E000E0320EA6E080EEC6E9B
:102E0000ED52AC0EEF6EF5EF22F0D8909C35026ECD
:102E10009D35036E0250870FE96E000E0320EA6EA7
:102E2000080EEC6EED52CA0EEF6EF5EF22F0D89060
:102E30009C35026E9D35036E0250870FE96E000EC1
:102E40000320EA6E080EEC6EED52E80EEF6EF5EF21
:102E500022F0D8909C35026E9D35036E0250870F8C
:102E6000E96E000E0320EA6E090EEC6EED52060EBE
:102E7000EF6EF5EF22F0D8909C35026E9D35036E13
:102E80000250870FE96E000E0320EA6E090EEC6E09
:102E9000ED52240EEF6EF5EF22F0D8909C35026EC5
:102EA0009D35036E0250870FE96E000E0320EA6E17
:102EB000090EEC6EED52420EEF6EF5EF22F0D89057
:102EC0009C35026E9D35036E0250870FE96E000E31
:102ED0000320EA6E090EEC6EED52600EEF6EF5EF18
:102EE00022F0D8909C35026E9D35036E0250870FFC
:102EF000E96E000E0320EA6E090EEC6EED527E0EB6
:102F0000EF6EF5EF22F0D8909C35026E9D35036E82
:102F10000250870FE96E000E0320EA6E090EEC6E78
:102F2000ED529C0EEF6EF5EF22F0D8909C35026EBC
:102F30009D35036E0250870FE96E000E0320EA6E86
:102F4000090EEC6EED52BA0EEF6EF5EF22F0D8904E
:102F50009C35026E9D35036E0250870FE96E000EA0
:102F60000320EA6E090EEC6EED52D80EEF6EF5EF0F
:102F700022F0D8909C35026E9D35036E0250870F6B
:102F8000E96E000E0320EA6E090EEC6EED52F60EAD
:102F9000EF6EF5EF22F0D8909C35026E9D35036EF2
:102FA0000250870FE96E000E0320EA6E0A0EEC6EE7
:102FB000ED52140EEF6EF5EF22F0D8909C35026EB4
:102FC0009D35036E0250870FE96E000E0320EA6EF6
:102FD0000A0EEC6EED52320EEF6EF5EF22F0D89045
:102FE0009C35026E9D35036E0250870FE96E000E10
:102FF0000320EA6E0A0EEC6EED52500EEF6EF5EF06
:1030000022F0D8909C35026E9D35036E0250870FDA
:10301000E96E000E0320EA6E0A0EEC6EED526E0EA3
:10302000EF6EF5EF22F0D8909C35026E9D35036E61
:103030000250870FE96E000E0320EA6E0A0EEC6E56
:10304000ED528C0EEF6EF5EF22F0D8909C35026EAB
:103050009D35036E0250870FE96E000E0320EA6E65
:103060000A0EEC6EED52AA0EEF6EF5EF22F0D8903C
:103070009C35026E9D35036E0250870FE96E000E7F
:103080000320EA6E0A0EEC6EED52C80EEF6EF5EFFD
:1030900022F0D8909C35026E9D35036E0250870F4A
:1030A000E96E000E0320EA6E0A0EEC6EED52E60E9B
:1030B000EF6EF5EF22F0D8909C35026E9D35036ED1
:1030C0000250870FE96E000E0320EA6E0B0EEC6EC5
:1030D000ED52040EEF6EF5EF22F0D8909C35026EA3
:1030E0009D35036E0250870FE96E000E0320EA6ED5
:1030F0000B0EEC6EED52220EEF6EF5EF22F0D89033
:103100009C35026E9D35036E0250870FE96E000EEE
:103110000320EA6E0B0EEC6EED52400EEF6EF5EFF3
:1031200022F0D8909C35026E9D35036E0250870FB9
:10313000E96E000E0320EA6E0B0EEC6EED525E0E91
:10314000EF6EF5EF22F0D8909C35026E9D35036E40
:103150000250870FE96E000E0320EA6E0B0EEC6E34
:10316000ED527C0EEF6EF5EF22F0D8909C35026E9A
:103170009D35036E0250870FE96E000E0320EA6E44
:103180000B0EEC6EED529A0EEF6EF5EF22F0D8902A
:103190009C35026E9D35036E0250870FE96E000E5E
:1031A0000320EA6E0B0EEC6EED52B80EEF6EF5EFEB
:1031B00022F0D8909C35026E9D35036E0250870F29
:1031C000E96E000E0320EA6E0B0EEC6EED52D60E89
:1031D000EF6EF5EF22F0D8909C35026E9D35036EB0
:1031E0000250870FE96E000E0320EA6E0B0EEC6EA4
:1031F000ED52F40EEF6EF5EF22F0D8909C35026E92
:103200009D35036E0250870FE96E000E0320EA6EB3
:103210000C0EEC6EED52120EEF6EF5EF22F0D89020
:103220009C35026E9D35036E0250870FE96E000ECD
:103230000320EA6E0C0EEC6EED52300EEF6EF5EFE1
:1032400022F0D8909C35026E9D35036E0250870F98
:10325000E96E000E0320EA6E0C0EEC6EED524E0E7F
:10326000EF6EF5EF22F0D8909C35026E9D35036E1F
:103270000250870FE96E000E0320EA6E0C0EEC6E12
:10328000ED526C0EEF6EF5EF22F0D8909C35026E89
:103290009D35036E0250870FE96E000E0320EA6E23
:1032A0000C0EEC6EED528A0EEF6EF5EF22F0D89018
:1032B0009C35026E9D35036E0250870FE96E000E3D
:1032C0000320EA6E0C0EEC6EED52A80EEF6EF5EFD9
:1032D00022F0D8909C35026E9D35036E0250870F08
:1032E000E96E000E0320EA6E0C0EEC6EED52C60E77
:1032F000EF6EF5EF22F0D8909C35026E9D35036E8F
:103300000250870FE96E000E0320EA6E0C0EEC6E81
:10331000ED52E40EEF6EF5EF22F0D8909C35026E80
:103320009D35036E0250870FE96E000E0320EA6E92
:103330000D0EEC6EED52020EEF6EF5EF22F0D8900E
:103340009C35026E9D35036E0250870FE96E000EAC
:103350000320EA6E0D0EEC6EED52200EEF6EF5EFCF
:1033600022F0D8909C35026E9D35036E0250870F77
:10337000E96E000E0320EA6E0D0EEC6EED523E0E6D
:10338000EF6EF5EF22F0D8909C35026E9D35036EFE
:103390000250870FE96E000E0320EA6E0D0EEC6EF0
:1033A000ED525C0EEF6EF5EF22F0D8909C35026E78
:1033B0009D35036E0250870FE96E000E0320EA6E02
:1033C0000D0EEC6EED527A0EEF6EF5EF22F0D89006
:1033D0009C35026E9D35036E0250870FE96E000E1C
:1033E0000320EA6E0D0EEC6EED52980EEF6EF5EFC7
:1033F00022F0D8909C35026E9D35036E0250870FE7
:10340000E96E000E0320EA6E0D0EEC6EED52B60E64
:10341000EF6EF5EF22F0D8909C35026E9D35036E6D
:103420000250870FE96E000E0320EA6E0D0EEC6E5F
:10343000ED52D40EEF6EF5EF22F0D8909C35026E6F
:103440009D35036E0250870FE96E000E0320EA6E71
:103450000D0EEC6EED52F20EEF6EF5EF22F0D890FD
:103460009C35026E9D35036E0250870FE96E000E8B
:103470000320EA6E0E0EEC6EED52100EEF6EF5EFBD
:1034800022F0D8909C35026E9D35036E0250870F56
:10349000E96E000E0320EA6E0E0EEC6EED522E0E5B
:1034A000EF6EF5EF22F0D8909C35026E9D35036EDD
:1034B0000250870FE96E000E0320EA6E0E0EEC6ECE
:1034C000ED524C0EEF6EF5EF22F0D8909C35026E67
:1034D0009D35036E0250870FE96E000E0320EA6EE1
:1034E0000E0EEC6EED526A0EEF6EF5EF22F0D890F4
:1034F0009C35026E9D35036E0250870FE96E000EFB
:103500000320EA6E0E0EEC6EED52880EEF6EF5EFB4
:1035100022F0D8909C35026E9D35036E0250870FC5
:10352000E96E000E0320EA6E0E0EEC6EED52A60E52
:10353000EF6EF5EF22F0D8909C35026E9D35036E4C
:103540000250870FE96E000E0320EA6E0E0EEC6E3D
:10355000ED52C40EEF6EF5EF22F0D8909C35026E5E
:103560009D35036E0250870FE96E000E0320EA6E50
:103570000E0EEC6EED52E20EEF6EF5EF22F0D890EB
:103580009C35026E9D35036E0250870FE96E000E6A
:103590000320EA6E0F0EEC6EED52EF6AF5EF22F0AB
:1035A000D8909C35026E9D35036E0250870FE96EF0
:1035B000000E0320EA6E0F0EEC6EED521E0EEF6E43
:1035C000F5EF22F0D8909C35026E9D35036E0250C7
:1035D000870FE96E000E0320EA6E0F0EEC6EED52BF
:1035E0003C0EEF6EF5EF22F0D8909C35026E9D35C3
:1035F000036E0250870FE96E000E0320EA6E0F0E75
:10360000EC6EED525A0EEF6EF5EF22F0D8909C352D
:10361000026E9D35036E0250870FE96E000E032087
:10362000EA6E0F0EEC6EED52780EEF6EF5EF22F0B3
:10363000D8909C35026E9D35036E0250870FE96E5F
:10364000000E0320EA6E0F0EEC6EED52960EEF6E3A
:10365000F5EF22F0D8909C35026E9D35036E025036
:10366000870FE96E000E0320EA6E0F0EEC6EED522E
:10367000B40EEF6EF5EF22F0D8909C35026E9D35BA
:10368000036E0250870FE96E000E0320EA6E0F0EE4
:10369000EC6EED52D20EEF6EF5EF22F0D8909C3525
:1036A000026E9D35036E0250870FE96E000E0320F7
:1036B000EA6E0F0EEC6EED52F00EEF6EF5EF22F0AB
:1036C000D8909C35026E9D35036E0250870FE96ECF
:1036D000000E0320EA6E100EEC6EED520E0EEF6E31
:1036E000F5EF22F0D8909C35026E9D35036E0250A6
:1036F000870FE96E000E0320EA6E100EEC6EED529D
:103700002C0EEF6EF5EF22F0D8909C35026E9D35B1
:10371000036E0250870FE96E000E0320EA6E100E52
:10372000EC6EED524A0EEF6EF5EF22F0D8909C351C
:10373000026E9D35036E0250870FE96E000E032066
:10374000EA6E100EEC6EED52680EEF6EF5EF22F0A1
:10375000D8909C35026E9D35036E0250870FE96E3E
:10376000000E0320EA6E100EEC6EED52860EEF6E28
:10377000F5EF22F0D8909C35026E9D35036E025015
:10378000870FE96E000E0320EA6E100EEC6EED520C
:10379000A40EEF6EF5EF22F0D8909C35026E9D35A9
:1037A000036E0250870FE96E000E0320EA6E100EC2
:1037B000EC6EED52C20EEF6EF5EF22F0D8909C3514
:1037C000026E9D35036E0250870FE96E000E0320D6
:1037D000EA6E100EEC6EED52E00EEF6EF5EF22F099
:1037E000D8909C35026E9D35036E0250870FE96EAE
:1037F000000E0320EA6E100EEC6EED52FE0EEF6E20
:10380000F5EF22F0D8909C35026E9D35036E025084
:10381000870FE96E000E0320EA6E110EEC6EED527A
:103820001C0EEF6EF5EF22F0D8909C35026E9D35A0
:10383000036E0250870FE96E000E0320EA6E110E30
:10384000EC6EED523A0EEF6EF5EF22F0D8909C350B
:10385000026E9D35036E0250870FE96E000E032045
:10386000EA6E110EEC6EED52580EEF6EF5EF22F08F
:10387000D8909C35026E9D35036E0250870FE96E1D
:10388000000E0320EA6E110EEC6EED52760EEF6E16
:10389000F5EF22F0D8909C35026E9D35036E0250F4
:1038A000870FE96E000E0320EA6E110EEC6EED52EA
:1038B000940EEF6EF5EF22F0D8909C35026E9D3598
:1038C000036E0250870FE96E000E0320EA6E110EA0
:1038D000EC6EED52B20EEF6EF5EF22F0D8909C3503
:1038E000026E9D35036E0250870FE96E000E0320B5
:1038F000EA6E110EEC6EED52D00EEF6EF5EF22F087
:10390000D8909C35026E9D35036E0250870FE96E8C
:10391000000E0320EA6E110EEC6EED52EE0EEF6E0D
:10392000F5EF22F0D8909C35026E9D35036E025063
:10393000870FE96E000E0320EA6E120EEC6EED5258
:103940000C0EEF6EF5EF22F0D8909C35026E9D358F
:10395000036E0250870FE96E000E0320EA6E120E0E
:10396000EC6EED522A0EEF6EF5EF22F0D8909C35FA
:10397000026E9D35036E0250870FE96E000E032024
:10398000EA6E120EEC6EED52480EEF6EF5EF22F07D
:10399000D8909C35026E9D35036E0250870FE96EFC
:1039A000000E0320EA6E120EEC6EED52660EEF6E04
:1039B000F5EF22F0D8909C35026E9D35036E0250D3
:1039C000870FE96E000E0320EA6E120EEC6EED52C8
:1039D000840EEF6EF5EF22F0D8909C35026E9D3587
:1039E000036E0250870FE96E000E0320EA6E120E7E
:1039F000EC6EED52A20EEF6EF5EF22F0D8909C35F2
:103A0000026E9D35036E0250870FE96E000E032093
:103A1000EA6E120EEC6EED52C00EEF6EF5EF22F074
:103A2000D8909C35026E9D35036E0250870FE96E6B
:103A3000000E0320EA6E120EEC6EED52DE0EEF6EFB
:103A4000F5EF22F0D8909C35026E9D35036E025042
:103A5000870FE96E000E0320EA6E120EEC6EED5237
:103A6000FC0EEF6EF5EF22F0D8909C35026E9D357E
:103A7000036E0250870FE96E000E0320EA6E130EEC
:103A8000EC6EED521A0EEF6EF5EF22F0D8909C35E9
:103A9000026E9D35036E0250870FE96E000E032003
:103AA000EA6E130EEC6EED52380EEF6EF5EF22F06B
:103AB000D8909C35026E9D35036E0250870FE96EDB
:103AC000000E0320EA6E130EEC6EED52560EEF6EF2
:103AD000F5EF22F0D8909C35026E9D35036E0250B2
:103AE000870FE96E000E0320EA6E130EEC6EED52A6
:103AF000740EEF6EF5EF22F0D8909C35026E9D3576
:103B0000036E0250870FE96E000E0320EA6E130E5B
:103B1000EC6EED52920EEF6EF5EF22F0D8909C35E0
:103B2000026E9D35036E0250870FE96E000E032072
:103B3000EA6E130EEC6EED52B00EEF6EF5EF22F062
:103B4000D8909C35026E9D35036E0250870FE96E4A
:103B5000000E0320EA6E130EEC6EED52CE0EEF6EE9
:103B6000F5EF22F0D8909C35026E9D35036E025021
:103B7000870FE96E000E0320EA6E130EEC6EED5215
:103B8000EC0EEF6EF5EF22F0D8909C35026E9D356D
:103B9000036E0250870FE96E000E0320EA6E140ECA
:103BA000EC6EED520A0EEF6EF5EF22F0D8909C35D8
:103BB000026E9D35036E0250870FE96E000E0320E2
:103BC000EA6E140EEC6EED52280EEF6EF5EF22F059
:103BD000D8909C35026E9D35036E0250870FE96EBA
:103BE000000E0320EA6E140EEC6EED52460EEF6EE0
:103BF000F5EF22F0D8909C35026E9D35036E025091
:103C0000870FE96E000E0320EA6E140EEC6EED5283
:103C1000640EEF6EF5EF22F0D8909C35026E9D3564
:103C2000036E0250870FE96E000E0320EA6E140E39
:103C3000EC6EED52820EEF6EF5EF22F0D8909C35CF
:103C4000026E9D35036E0250870FE96E000E032051
:103C5000EA6E140EEC6EED52A00EEF6EF5EF22F050
:103C6000D8909C35026E9D35036E0250870FE96E29
:103C7000000E0320EA6E140EEC6EED52BE0EEF6ED7
:103C8000F5EF22F0D8909C35026E9D35036E025000
:103C9000870FE96E000E0320EA6E140EEC6EED52F3
:103CA000DC0EEF6EF5EF22F0D8909C35026E9D355C
:103CB000036E0250870FE96E000E0320EA6E140EA9
:103CC000EC6EED52FA0EEF6EF5EF22F0D8909C35C7
:103CD000026E9D35036E0250870FE96E000E0320C1
:103CE000EA6E150EEC6EED52180EEF6EF5EF22F047
:103CF000D8909C35026E9D35036E0250870FE96E99
:103D0000000E0320EA6E150EEC6EED52360EEF6ECD
:103D1000F5EF22F0D8909C35026E9D35036E02506F
:103D2000870FE96E000E0320EA6E150EEC6EED5261
:103D3000540EEF6EF5EF22F0D8909C35026E9D3553
:103D4000036E0250870FE96E000E0320EA6E150E17
:103D5000EC6EED52720EEF6EF5EF22F0D8909C35BE
:103D6000026E9D35036E0250870FE96E000E032030
:103D7000EA6E150EEC6EED52900EEF6EF5EF22F03E
:103D8000D8909C35026E9D35036E0250870FE96E08
:103D9000000E0320EA6E150EEC6EED52AE0EEF6EC5
:103DA000F5EF22F0D8909C35026E9D35036E0250DF
:103DB000870FE96E000E0320EA6E150EEC6EED52D1
:103DC000CC0EEF6EF5EF22F0D8909C35026E9D354B
:103DD000036E0250870FE96E000E0320EA6E150E87
:103DE000EC6EED52EA0EEF6EF5EF22F0D8909C35B6
:103DF000026E9D35036E0250870FE96E000E0320A0
:103E0000EA6E160EEC6EED52080EEF6EF5EF22F034
:103E1000D8909C35026E9D35036E0250870FE96E77
:103E2000000E0320EA6E160EEC6EED52260EEF6EBB
:103E3000F5EF22F0D8909C35026E9D35036E02504E
:103E4000870FE96E000E0320EA6E160EEC6EED523F
:103E5000440EEF6EF5EF22F0D8909C35026E9D3542
:103E6000036E0250870FE96E000E0320EA6E160EF5
:103E7000EC6EED52620EEF6EB8D3D8909C35026EA8
:103E80009D35036E0250870FE96E000E0320EA6E27
:103E9000160EEC6EED52800EEF6EA7D3D8909C35C7
:103EA000026E9D35036E0250870FE96E000E0320EF
:103EB000EA6E160EEC6EED529E0EEF6E96D3D89013
:103EC0009C35026E9D35036E0250870FE96E000E21
:103ED0000320EA6E160EEC6EED52BC0EEF6E85D32B
:103EE000D8909C35026E9D35036E0250870FE96EA7
:103EF000000E0320EA6E160EEC6EED52DA0EEF6E37
:103F000074D3D8909C35026E9D35036E0250870F96
:103F1000E96E000E0320EA6E160EEC6EED52F80EFE
:103F2000EF6E63D3D8909C35026E9D35036E0250C0
:103F3000870FE96E000E0320EA6E170EEC6EED524D
:103F4000160EEF6E52D3D8909C35026E9D35036EDF
:103F50000250870FE96E000E0320EA6E170EEC6E1A
:103F6000ED52340EEF6E41D3D8909C35026E9D35E4
:103F7000036E0250870FE96E000E0320EA6E170EE3
:103F8000EC6EED52520EEF6E30D3D8909C35026E2F
:103F90009D35036E0250870FE96E000E0320EA6E16
:103FA000170EEC6EED52700EEF6E1FD3D8909C354D
:103FB000026E9D35036E0250870FE96E000E0320DE
:103FC000EA6E170EEC6EED528E0EEF6E0ED3D89099
:103FD0009C35026E9D35036E0250870FE96E000E10
:103FE0000320EA6E170EEC6EED52AC0EEF6EFDD2B2
:103FF000D8909C35026E9D35036E0250870FE96E96
:10400000000E0320EA6E170EEC6EED52CA0EEF6E34
:10401000ECD2D8909C35026E9D35036E0250870F0E
:10402000E96E000E0320EA6E170EEC6EED52E80EFC
:10403000EF6EDBD2D8909C35026E9D35036E025038
:10404000870FE96E000E0320EA6E180EEC6EED523B
:10405000060EEF6ECAD2D8909C35026E9D35036E67
:104060000250870FE96E000E0320EA6E180EEC6E08
:10407000ED52240EEF6EB9D2D8909C35026E9D356C
:10408000036E0250870FE96E000E0320EA6E180ED1
:10409000EC6EED52420EEF6EA8D2D8909C35026EB7
:1040A0009D35036E0250870FE96E000E0320EA6E05
:1040B000180EEC6EED52600EEF6E97D2D8909C35D4
:1040C000026E9D35036E0250870FE96E000E0320CD
:1040D000EA6E180EEC6EED527E0EEF6E86D2D89020
:1040E0009C35026E9D35036E0250870FE96E000EFF
:1040F0000320EA6E180EEC6EED529C0EEF6E75D238
:10410000D8909C35026E9D35036E0250870FE96E84
:10411000000E0320EA6E180EEC6EED52BA0EEF6E32
:1041200064D2D8909C35026E9D35036E0250870F85
:10413000E96E000E0320EA6E180EEC6EED52D80EFA
:10414000EF6E53D2D8909C35026E9D35036E0250AF
:10415000870FE96E000E0320EA6E180EEC6EED522A
:10416000F60EEF6E42D2D8909C35026E9D35036EEE
:104170000250870FE96E000E0320EA6E190EEC6EF6
:10418000ED52140EEF6E31D2D8909C35026E9D35F3
:10419000036E0250870FE96E000E0320EA6E190EBF
:1041A000EC6EED52320EEF6E20D2D8909C35026E3E
:1041B0009D35036E0250870FE96E000E0320EA6EF4
:1041C000190EEC6EED52500EEF6E0FD2D8909C355A
:1041D000026E9D35036E0250870FE96E000E0320BC
:1041E000EA6E190EEC6EED526E0EEF6EFED1D890A7
:1041F0009C35026E9D35036E0250870FE96E000EEE
:104200000320EA6E190EEC6EED528C0EEF6EEDD1BE
:10421000D8909C35026E9D35036E0250870FE96E73
:10422000000E0320EA6E190EEC6EED52AA0EEF6E30
:10423000DCD1D8909C35026E9D35036E0250870FFD
:10424000E96E000E0320EA6E190EEC6EED52C80EF8
:10425000EF6ECBD1D8909C35026E9D35036E025027
:10426000870FE96E000E0320EA6E190EEC6EED5218
:10427000E60EEF6EBAD1D8909C35026E9D35036E76
:104280000250870FE96E000E0320EA6E1A0EEC6EE4
:10429000ED52040EEF6EA9D1D8909C35026E9D357B
:1042A000036E0250870FE96E000E0320EA6E1A0EAD
:1042B000EC6EED52220EEF6E98D1D8909C35026EC6
:1042C0009D35036E0250870FE96E000E0320EA6EE3
:1042D0001A0EEC6EED52400EEF6E87D1D8909C35E1
:1042E000026E9D35036E0250870FE96E000E0320AB
:1042F000EA6E1A0EEC6EED525E0EEF6E76D1D8902D
:104300009C35026E9D35036E0250870FE96E000EDC
:104310000320EA6E1A0EEC6EED527C0EEF6E65D144
:10432000D8909C35026E9D35036E0250870FE96E62
:10433000000E0320EA6E1A0EEC6EED529A0EEF6E2E
:1043400054D1D8909C35026E9D35036E0250870F74
:10435000E96E000E0320EA6E1A0EEC6EED52B80EF6
:10436000EF6E43D1D8909C35026E9D35036E02509E
:10437000870FE96E000E0320EA6E1A0EEC6EED5206
:10438000D60EEF6E32D1D8909C35026E9D35036EFD
:104390000250870FE96E000E0320EA6E1A0EEC6ED3
:1043A000ED52F40EEF6E21D1D8909C35026E9D3502
:1043B000036E0250870FE96E000E0320EA6E1B0E9B
:1043C000EC6EED52120EEF6E10D1D8909C35026E4D
:1043D0009D35036E0250870FE96E000E0320EA6ED2
:1043E0001B0EEC6EED52300EEF6EFFD0D8909C3568
:1043F000026E9D35036E0250870FE96E000E03209A
:10440000EA6E1B0EEC6EED524E0EEF6EEED0D890B3
:104410009C35026E9D35036E0250870FE96E000ECB
:104420000320EA6E1B0EEC6EED526C0EEF6EDDD0CB
:10443000D8909C35026E9D35036E0250870FE96E51
:10444000000E0320EA6E1B0EEC6EED528A0EEF6E2C
:10445000CCD0D8909C35026E9D35036E0250870FEC
:10446000E96E000E0320EA6E1B0EEC6EED52A80EF4
:10447000EF6EBBD0D8909C35026E9D35036E025016
:10448000870FE96E000E0320EA6E1B0EEC6EED52F4
:10449000C60EEF6EAAD0D8909C35026E9D35036E85
:1044A0000250870FE96E000E0320EA6E1B0EEC6EC1
:1044B000ED52E40EEF6E99D0D8909C35026E9D358A
:1044C000036E0250870FE96E000E0320EA6E1C0E89
:1044D000EC6EED52020EEF6E88D0D8909C35026ED5
:1044E0009D35036E0250870FE96E000E0320EA6EC1
:1044F0001C0EEC6EED52200EEF6E77D0D8909C35EE
:10450000026E9D35036E0250870FE96E000E032088
:10451000EA6E1C0EEC6EED523E0EEF6E66D0D89039
:104520009C35026E9D35036E0250870FE96E000EBA
:104530000320EA6E1C0EEC6EED525C0EEF6E55D051
:10454000D8909C35026E9D35036E0250870FE96E40
:10455000000E0320EA6E1C0EEC6EED527A0EEF6E2A
:1045600044D0D8909C35026E9D35036E0250870F63
:10457000E96E000E0320EA6E1C0EEC6EED52980EF2
:10458000EF6E33D0D8909C35026E9D35036E02508D
:10459000870FE96E000E0320EA6E1C0EEC6EED52E2
:1045A000B60EEF6E22D0D8909C35026E9D35036E0C
:1045B0000250870FE96E000E0320EA6E1C0EEC6EAF
:1045C000ED52D40EEF6E11D0D8909C35026E9D3511
:1045D000036E0250870FE96E000E0320EA6E1C0E78
:1045E000EC6EED52F20EEF6E00D0B2EF0DF0030064
:020000040030CA
:0E000000240E3E1E008381000FC00FE00F4053
:00000001FF
